:020000040000FA
:42000000FFFF62F73300FFFFFFFFFFFFFFFFFFFFFFFFFFFFFFFFFFFFFFFFFFFFFFFFFFFFFFFFFFFFFFFFFFFFFFFFFFFFFFFFFFFFFFFFFFFFFFFFFFFFFFFFFFFFFFFFFFFFFFFF70
:42004200A00C9881325006CA40190053600A4C81A9325506CA401928034C80613001000000000006984013001324830C900132400618061360022002648001300006C00014FE3E
:420084000015A00254800A50012A800A50012A4005B4800A50012A4005A8002DA00200000000000950012A800E780117E0025C800BD0022A400550012A400248000920013CFE56
:4200C6000004800010000240000800024000080001300002400008000100000000000000000000000000000000000000000000000000000000000000000000000000000010FC48
:42010800000000000000000000000000000000000000000000000000000000000000000000000000000000000000000000000000000000000000000000000000000000003CFE7B
:42014A0040012800048000100002000800012000048680001480024000000000000000000000000000000000080800000000000000000000000000000000000000000000FCFF60
:42018C0000000000148002200002004244800810011480020000004000000000000000000000000000000000000000000000000000000000000000000000000000000000E0FFA5
:4201CE00001001000000000000000000000000000000000000110000000000000000000000000000000000000000000000000000000000000000000000000000000000003CFE93
:42021000000000000000000000000000000000000000000000000000000000000000000000000000000000000000000000000000000000000000000000000000000000003CFE72
:42025200600000000000000000000000000000000000000006000000000000000000000000000000000000000000000000000000000000000000000000000000000000003CFECA
:42029400200000000000000000000000000000000000000002000000000000000000000000000000000000000000000000000000000000000000000000000000000000003CFECC
:4202D600804100000000000000000000000000000000000018040000000000000000000000000000000000000000000000000000000000000000000000000000000000003CFECF
:42031800E0010000000000000000000000000000000000001E000000000000000000000000000000000000000000000000000000000000000000000000000000000000003CFE6A
:42035A00800100000000000000000000000000000000000018000000000000000000000000000000000000000000000000000000000000000000000000000000000000003CFE8E
:42039C00800100000000000000000000000000000000000018000000000000000000000000000000000000000000000000000000000000000000000000000000000000003CFE4C
:4203DE00000004010000001A000000000000000000000000000000000000000000000000000000000000000000000000000000000000000000000000000000000000000072FE4E
:4204200000000008000000000000000000000000000000000000000000000000000000000000000000000000000000000000000000000000000000000000000000000000BCFED8
:4204620000001C080000001E00000000000000000000000000000000000000000000000000000000000000000000000000000000000000000000000000000000000000005CFDBD
:4204A4000800040000000002040000000000000000000000000000000000000000000000000000000000000000000000000000000000000000000000000000000000008005FD82
:4204E60000003002000000000500000000000000000000000000000000000000000000000000000000000000000000000000000000000000000000000000000000000080E0FC41
:4205280000003C080000001E00000000000000000000000000000000000000000000000000000000000000000000000000000000000000000000000000000000000000007CFFB4
:42056A000400300800000000000000000000000000000000000000000000000000000000000000000000000000000000000000000000000000000000000000000000008055FC42
:4205AC000000940000000040040000000000000000000000000000000000000000000000000000000000000000000000000000000000000000000000000000000000000064FFD2
:4205EE00000000200000000200000000000000000000000000000000000000000000000000000000000000000000000000000000000000000000000000000000000000001CFE8F
:42063000000000000000000000000000000000000000000000000000000000000000000000000000000000000000000000000000000000000000000000000000000000003CFE4E
:4206720000003C000000001E0000000000000000000000000000000000000000000000000000000000000000000000000000000000000000000000000000000000000000FCFFF1
:4206B400040034000000001A000000000000000000000000000000000000000000000000000000000000000000000000000000000000000000000000000000000000000021FE93
:4206F6000C00B00000000018050000000000000000000000000000000000000000000000000000000000000000000000000000000000000000000000000000000000000098FC55
:4207380000003C080000001E00000000000000000000000000000000000000000000000000000000000000000000000000000000000000000000000000000000000000007CFFA2
:42077A0008000008000000000000000000000000000000000000000000000000000000000000000000000000000000000000000000000000000000000000000000000080B4FEFB
:4207BC000000000100000040040000000000000000000000000000000000000000000000000000000000000000000000000000000000000000000000000000000000000028FE90
:4207FE00001035000000008A0000000000000000000000000000000000000000000000000000000000000000000000000000000000000000000000000000000000000000D2FC1C
:420840000000000000000010040000000000000000000000000000000000000000000000000000000000000000000000000000000000000000000000000000000000000068FEFC
:4208820060003C00000000060400000000000000000000000000000000000000000000000000000000000000000000000000000000000000000000000000000000000000E4FDAD
:4208C4002800040A000000420000000000000000000000000000000000000000000000000000000000000000000000000000000000000000000000000000000000000080A1FF5A
:420906008051000A00000088040000000000000000000000000000000000000000000000000000000000000000000000000000000000000000000000000000000000008010FFB9
:42094800E0013C000000000E000000000000000000000000000000000000000000000000000000000000000000000000000000000000000000000000000000000000000030FC16
:42098A008401300800000000040000000000000000000000000000000000000000000000000000000000000000000000000000000000000000000000000000000000008089FD64
:4209CC008001840000000080000000000000000000000000000000000000000000000000000000000000000000000000000000000000000000000000000000000000000068FFFD
:420A0E00000004000000001A000000000000000000000000000000000000000000000000000000000000000000000000000000000000000000000000000000000000000062FE28
:420A50000000000000000018000000000000000000000000000000000000000000000000000000000000000000000000000000000000000000000000000000000000000024FE2A
:420A9200000030000000001E000000000000000000000000000000000000000000000000000000000000000000000000000000000000000000000000000000000000000030FFA5
:420AD400040030000000001A0000000000000000000000000000000000000000000000000000000000000000000000000000000000000000000000000000000000000080EDFE27
:420B16000C003002000000800400000000000000000000000000000000000000000000000000000000000000000000000000000000000000000000000000000000000080A0FDBE
:420B580000003C0800000006000000000000000000000000000000000000000000000000000000000000000000000000000000000000000000000000000000000000000064FFAE
:420B9A000800000000000000000000000000000000000000000000000000000000000000000000000000000000000000000000000000000000000000000000000000008025FF6D
:420BDC0000008008000000000000000000000000000000000000000000000000000000000000000000000000000000000000000000000000000000000000000000000000B4FE9D
:420C1E00000004000000001A000000000000000000000000000000000000000000000000000000000000000000000000000000000000000000000000000000000000000062FE16
:420C6000000000000000000000000000000000000000000000000000000000000000000000000000000000000000000000000000000000000000000000000000000000003CFE18
:420CA20000003C00000000060400000000000000000000000000000000000000000000000000000000000000000000000000000000000000000000000000000000000000A0FF2B
:420CE400080034000000005A000000000000000000000000000000000000000000000000000000000000000000000000000000000000000000000000000000000000008029FE91
:420D26000000300A00000000040000000000000000000000000000000000000000000000000000000000000000000000000000000000000000000000000000000000008060FD70
:420D680000003C00000000060000000000000000000000000000000000000000000000000000000000000000000000000000000000000000000000000000000000000000E4FF24
:420DAA000400000800000000040000000000000000000000000000000000000000000000000000000000000000000000000000000000000000000000000000000000008021FF57
:420DEC000000840000000000010000000000000000000000000000000000000000000000000000000000000000000000000000000000000000000000000000000000000070FFD1
:420E2E008009340000C00402000000000000000000000000000000000000000000000000000000000000000000000000000000000000000000000000000000000000000096FC6D
:420E700000803000000040000000000000000000000000000000000000000000000000000000000000000000000000000000000000000000000000000000000000000000C8FD8B
:420EB200E0013C0000F00000000000000000000000000000000000000000000000000000000000000000000000000000000000000000000000000000000000000000000020FDD4
:420EF4002484340000101400050000000000000000000000000000000000000000000000000000000000000000000000000000000000000000000000000000000000008001FF37
:420F36000C00000A00000080040000000000000000000000000000000000000000000000000000000000000000000000000000000000000000000000000000000000008010FE51
:420F7800E0010C0000F00006000000000000000000000000000000000000000000000000000000000000000000000000000000000000000000000000000000000000000034FC24
:420FBA000800000000000000040000000000000000000000000000000000000000000000000000000000000000000000000000000000000000000000000000000000008061FF09
:420FFC008001040000C000580000000000000000000000000000000000000000000000000000000000000000000000000000000000000000000000000000000000000000B4FF63
:42103E008009302000008802000000000000000000000000980000000000000000000000000000000000000000000000000000000000000000000000000000000000000024FD54
:42108000008030000000000000000000000000000000000000080000000000000000000000000000000000000000000000000000000000000000000000000000000000000CFD6D
:4210C200E0813C00003000000000000000000000000000001E08000000000000000000000000000000000000000000000000000000000000000000000000000000000000F0FE0B
:421104002810340000100000040000000000000000000000420000000000000000000000000000000000000000000000000000000000000000000000000000000000000099FD51
:421146000000000800C02800050000000000000000000000000000000000000000000000000000000000000000000000000000000000000000000000000000000000000074FD01
:42118800E0010C0000F000060000000000000000000000001E00000000000000000000000000000000000000000000000000000000000000000000000000000000000000E8FF3D
:4211CA000400000000C000180000000000000000000000000000000000000000000000000000000000000000000000000000000000000000000000000000000000000080E0FEA9
:42120C008001000000C00040040000000000000000000000180000000000000000000000000000000000000000000000000000000000000000000000000000000000000034FED1
:42124E00000000000000000000000000000000000000000000000000000000000000000000000000000000000000000000000000000000000000000000000000000000001EFC44
:421290002000008000100002400008000120000480001000024000080001200004000000000010000240000800012000048000100002400008000120000480001000020070FC82
:4212D200000020000000000000000000000000000000000000000000000000000000000000000000000000000000000000000000000000000000000000000000000000001CFCA2
:4213140024000480001000024000080001200004800010000240000800012000040000000000100002400008000120000480001000024000080001200004800010000280EDFDF7
:421356000C0100000080000000000000000000000000000010000000000000000000000000000000000000000000000000000000000000000000000000000000000000807CFEBE
:421398000000008000000000400008000120000480001000004000080001200004000000000010000240000800012000048000100002400008000120000480001000020040FFDA
:4213DA000800200000000010000000000000000000000000000000000000000000000000000000000000000000000000000000000000000000000000000000000000008015FD07
:42141C002000048000100002400008000120000480001000024000080001200004000000000010000240000800012000048000100002400008000120000480001000020034FC2C
:42145E00000000000000000000000000000000000000000000000000000000000000000000000000000000000000000000000000000000000000000000000000000000003CFE12
:4214A000000000000000000000000000000000000000000000000000000000000000000000000000000000000000000000000000000000000000000000000000000000003CFED0
:4214E20000000000000000000000000000000000000000000800000000000000000000000000000000000000000000000000000000000000000000000000000000000000B4FE0E
:4215240000010000000000000000000000000000000000000000000000000000000000000000000000000000000000000000000000000000000000000000000000000080A4FF61
:42156600000000000000000000000000000000000000000000000000000000000000000000000000000000000000000000000000000000000000000000000000000000003CFE09
:4215A800000000000000000000000000000000000000000000000000000000000000000000000000000000000000000000000000000000000000000000000000000000003CFEC7
:4215EA00000000000000000000000000000000000000000000000000000000000000000000000000000000000000000000000000000000000000000000000000000000003CFE85
:42162C00000000000000000000000000000000000000000000000000000000000000000000000000000000000000000000000000000000000000000000000000000000003CFE42
:42166E00000000000000000000000000000000000000000000000000000000000000000000000000000000000000000000000000000000000000000000000000000000003CFE00
:4216B000000400000010020000000000000000000000000040000000000000000000000000000000000000000000000000000000000000000000000000000000000000000CFF97
:4216F200000000000000000000000000000000000000000000000000000000000000000000000000000000000000000000000000000000000000000000000000000000003CFE7C
:421734000000000000000000000000000000000000000000000000000000000000000000000000000000000000000000000000000000000000000000000000000000008096FC61
:42177600000000000000000000000000000000000000000000000000000000000000000000000000000000000000000000000000000000000000000000000000000010002CFFF6
:4217B800000000000000000000000000000000000000000000040000000000000000000000000000000000000000000000000000000000000000000000000000000000007CFE71
:4217FA000040000000000000000000000000000000000000001000000000000000000000000000000000000000000000000000000000000000000000000000000000040038FF22
:42183C000001000002000000000100000000400000000000000001000000020000000000000000000000000000000000000000000000000000000000000000000000000008FE1D
:42187E00000000000400000000020000000000010000000000000200000004000000000000000000000000000000000000000000000000000000000000000000000000006CFCB3
:4218C00080000000000000000000000000000000000000000000000000000000000000000000000000000000000000000000000000000000000000000000000000000000B4FEB4
:42190200000000000000000000000000000000000000000000000000000000000000000000000000000000000000000000000000000000000000000000000000000000003CFE69
:42194400000000000000000000000000000000000000000000000000000000000000000000000000000000000000000000000000000000000000000000000000000000003CFE27
:421986000000000000000000000000000000000000000000000000000000000000000000000000000000000000000000000000000000000000000000000000000000004078FE69
:4219C80080000000000000000000000000000000000000000000000000000000000000000000000000000000000000000000000000000000000000000000000000000000B4FEAB
:421A0A00000000000000000000000000000000000000000000000000000000000000000000000000000000000000000000000000000000000000000000000000000000003CFE60
:421A4C00000000000000000000000000000000000000000000000000000000000000000000000000000000000000000000000000000000000000000000000000000000001EFC3E
:421A8E00000000000000000000000000000000000000000000000000000000000000000000000000000000000000000000000000000000000000000000000000000000003CFEDC
:421AD000000000000000000000000000000000000000000000000000000000000000000000000000000000000000000000000000000000000000000000000000000000003CFE9A
:421B1200000000000000000000000000000000000000000000000000000000000000000000000000000000000000000000000000000000000000000000000000000000003CFE57
:421B5400000000000000000000000000000000000000000000000000000000000000000000000000000000000000000000000000000000000000000000000000000000003CFE15
:421B9600000000000000000000000000000000000000000000000000000000000000000000000000000000000000000000000000000000000000000000000000000000003CFED3
:421BD800000000000000000000000000000000000000000000000000000000000000000000000000000000000000000000000000000000000000000000000000000000003CFE91
:421C1A000000000000000000000000000000000000000000000000000000000000000000000000000000000000000000000000000000000000000000000000000000004069FFE0
:421C5C00000000000000000000000000000000000000000000000000000000000000000000000000000000000000000000000000000000000000000000000000000000003CFE0C
:421C9E000001000000800000000000000000000000000000100000000000000000000000000000000000000000000000000000000000000000000000000000000000000034FE41
:421CE000000000000000000000000000000000000000000000000000000000000000000000000000000000000000000000000000000000000000000000000000000000003CFE88
:421D2200000000000000000000000000000000000000000000000000000000000000000000000000000000000000000000000000000000000000000000000000000000003CFE45
:421D6400000000000000000000000000000000000000000000000000000000000000000000000000000000000000000000000000000000000000000000000000000000003CFE03
:421DA6000000000000000000000000000000000000000000000000000000000000000000000000000000400000000000000000000000000000000000000000000000000038FE85
:421DE800000000000000000000000000000000000000000000000000000000000000000000000000000000000000000000000000000000000000000000000000000000000FFDAD
:421E2A00004000060000000000000000000000000000000000000000000000000000000000000000000000010000000000000000000000000000000000000000000000000CFE25
:421E6C000008000400800008000000000000000000000000000000000000020000000000000000000000000000000000000000000000000000000000000000000000000074FC2E
:421EAE0000000000000000080000000000000000000000000000000000000800000000000000000000000000000000000000000000000000000000000000000000000000BCFE28
:421EF0000000000400400000000000000000000000000000000000000000000000000000000000000000000000000000000000000000000000000000000000000000000078FEF6
:421F3200000000000000000000000000000000000000000000000000000000000000000000000000000000000000000000000000000000000000000000000000000000003CFE33
:421F7400000000000000000000000000000000000000000000000000000000000000000000000000000000000000000000000000000000000000000000000000000000003CFEF1
:421FB6000000800000000000000000000000000000000000000000000000000000000000000000000000000000000000000000000000000000000000000000000000000034FE37
:421FF800000000000000000000000000000000000000000000000000000000000000000000000000000000000000000000000000000000000000000000000000000000003CFE6D
:42203A0008000000000000000000000000000000000000000000000000000000000000000000000000000000000000000000000000000000000000000000000000000000BCFEA2
:42207C00000000000000000000000000000000000000000000000000000000000000000000000000000000000000000000000000000000000000000000000000000000003CFEE8
:4220BE00000000000000000000000000000000000000000000000000000000000000000000000000000000000000000000000000000000000000000000000000000000003CFEA6
:42210000000000000000000000000000000000000000000000000000000000000000000000000000000000000000000000000000000000000000000000000000000000001EFC83
:42214200000000000000000000000000000000000000000000000000000000000000000000000000000000000000000000000000000000000000000000000000000000003CFE21
:42218400000000000000000000000000000000000000000000000000000000000000000000000000000000000000000000000000000000000000000000000000000000003CFEDF
:4221C600000000000000000000000000000000000000000000000000000000000000000000000000000000000000000000000000000000000000000000000000000000003CFE9D
:42220800000000000000000000000000000000000000000000000000000000000000000000000000000000000000000000000000000000000000000000000000000000003CFE5A
:42224A00000000000000000000000000000000000000000000000000000000000022000000000000000000000000000000000000000000000000000000000000000000001CFE16
:42228C00000000000000000000000000000000000000000000000000000000000000000000000000000000000000000000000000000000000000000000000000000000003CFED6
:4222CE00000000000000000000000000000000000000000000000000000000000C000000000000000000000000000000000000000000000000000000000000000000000030FE94
:422310000000000000000000000000000000000000000000000000000000000004000000000000000000000000000000000000000000000000000000000000000000000038FE51
:422352000000000000000000000000000000000000000000000000000000000030080000000000000000000000000000000000000000000000000000000000000000000084FE8F
:42239400000000000000000000000000000000000000000000000000000000003C000000000000000000000000000000000000000000000000000000000000000000000000FECD
:4223D600000000000000000000000000000000000000000000000000000000003000000000000000000000000000000000000000000000000000000000000000000000000CFE8B
:42241800000000000000000000000000000000000000000000000000000000003000000000000000000000000000000000000000000000000000000000000000000000000CFE48
:42245A00000000000000000000000000000000000000000000000000000000000000000000000000000000000000000000000000000000000000000000000000000000001EFC26
:42249C00000000000000000000000000000000000000000000000000000000000000000000000000000000000000000000000000000000000000000000000000000000003CFEC4
:4224DE00000000000000000000000000000000000000000000000000000000000000000000000000000000000000000000000000000000000000000000000000000000003CFE82
:422520000800000000000000000000000000000000000000000000000000000000000000000000000000000000000000000000000000000000000000000000000000008025FFCD
:4225620000000000000000000000000000000000000000000000000000000000000000000000000000000000000000000000000000000000000000000000000000000080B4FE05
:4225A400000000000000000000000000000000000000000000000000000000000000000000000000000000000000000000000000000000000000000000000000000000003CFEBB
:4225E60004000000000000000000000000000000000000000000000000000000000000000000000000000000000000000000000000000000000000000000000000000080E5FF4B
:42262800000000000000000000000000000000000000000000000000000000000000000000000000000000000000000000000000000000000000000000000000000000003CFE36
:42266A00000000000000000000000000000000000000000000000000000000000000000000000000000000000000000000000000000000000000000000000000000000003CFEF4
:4226AC00000000000000000000000000000000000000000000000000000000000000000000000000000000000000000000000000000000000000000000000000000000003CFEB2
:4226EE00000000000000000000000000000000000000000000000000000000000000000000000000000000000000000000000000000000000000000000000000000000003CFE70
:42273000040000000000000000000000000000000000000000000000000000000000000000000000000000000000000000000000000000000000000000000000000000006DFFF7
:422772000C000000000000000000000000000000000000000000000000000000000000000000000000000000000000000000000000000000000000000000000000000000FCFE1F
:4227B400000000000000000000000000000000000000000000000000000000000000000000000000000000000000000000000000000000000000000000000000000000003CFEA9
:4227F6000800000000000000000000000000000000000000000000000000000000000000000000000000000000000000000000000000000000000000000000000000008034FEE7
:42283800000000000000000000000000000000000000000000000000000000000000000000000000000000000000000000000000000000000000000000000000000000003CFE24
:42287A00000000000000000000000000000000000000000000000000000000000000000000000000000000000000000000000000000000000000000000000000000000003CFEE2
:4228BC00000000000000000000000000000000000000000000000000000000000000000000000000000000000000000000000000000000000000000000000000000000003CFEA0
:4228FE00000000000000000000000000000000000000000000000000000000000000000000000000000000000000000000000000000000000000000000000000000000003CFE5E
:42294000040000000000000000000000000000000000000000000000000000000000000000000000000000000000000000000000000000000000000000000000000000006DFFE5
:422982000C000000000000000000000000000000000000000000000000000000000000000000000000000000000000000000000000000000000000000000000000000000FCFE0D
:4229C400000000000000000000000000000000000000000000000000000000000000000000000000000000000000000000000000000000000000000000000000000000003CFE97
:422A06000800000000000000000000000000000000000000000000000000000000000000000000000000000000000000000000000000000000000000000000000000008034FED4
:422A4800000000000000000000000000000000000000000000000000000000000000000000000000000000000000000000000000000000000000000000000000000000003CFE12
:422A8A00000000000000000000000000000000000000000000000000000000000000000000000000000000000000000000000000000000000000000000000000000000001EFCF0
:422ACC00000000000000000000000000000000000000000000000000000000000000000000000000000000000000000000000000000000000000000000000000000000003CFE8E
:422B0E00000000000000000000000000000000000000000000000000000000000000000000000000000000000000000000000000000000000000000000000000000000003CFE4B
:422B500004000000000000000000000000000000000000000000000000000000000000000000000000000000000000000000000000000000000000000000000000000080E5FFDB
:422B92000C00000000000000000000000000000000000000000000000000000000000000000000000000000000000000000000000000000000000000000000000000008074FE03
:422BD400000000000000000000000000000000000000000000000000000000000000000000000000000000000000000000000000000000000000000000000000000000003CFE85
:422C16000800000000000000000000000000000000000000000000000000000000000000000000000000000000000000000000000000000000000000000000000000008025FFD0
:422C5800000000000000000000000000000000000000000000000000000000000000000000000000000000000000000000000000000000000000000000000000000000003CFE00
:422C9A00000000000000000000000000000000000000100000000000000000000000000000000000000000000000000000000000000000000000000000000000000000003CFFAD
:422CDC00000000000000000000000000000000000000000000000000000000000000000000000000000000000000000000000000000000000000000000000000000000003CFE7C
:422D1E00000000000000000000000000000000000000000000000000000000000000000000000000000000000000000000000000000000000000000000000000000000003CFE39
:422D6000040000000000000000000000000000000000000000000000000000000000000000000000000000000000000000000000000000000000000000000000000000006DFFC1
:422DA2000C0000000000000000000000000000000000C008000000000000000000000000000000000000000000000000000000000000000000000000000000000000000038FEE5
:422DE400000000000000000000000000000000000000F0400000000000000000000000000000000000000000000000000000000000000000000000000000000000000000B0FDD0
:422E2600080000000000000000000000000000000000C0000000000000000000000000000000000000000000000000000000000000000000000000000000000000000080F8FE2C
:422E6800000000000000000000000000000000000000C0000000000000000000000000000000000000000000000000000000000000000000000000000000000000000000F0FE7A
:422EAA00000000000000000000000000000000000000000000000000000000000000000000000000000000000000000000000000000000000000000000000000000000003CFEAC
:422EEC00000000000000000000000000000000000000000000000000000000000000000000000000000000000000000000000000000000000000000000000000000000003CFE6A
:422F2E00000000000000000000000000000000000000000000000000000000000000000000000000000000000000000000000000000000000000000000000000000000003CFE27
:422F700004000000000000000000000000000000000000000000000000000000000000000000000000000000000000000000000000000000000000000000000000000080E5FFB7
:422FB2000C00000000000000000000000000000000000000000000000000000000000000000000000000000000000000000000000000000000000000000000000000008074FEDF
:422FF400000000000000000000000000000000000000000000000000000000000000000000000000000000000000000000000000000000000000000000000000000000003CFE61
:423036000800000000000000000000000000000000000000000000000000000000000000000000000000000000000000000000000000000000000000000000000000008025FFAC
:42307800000000000000000000000000000000000000000000000000000000000000000000000000000000000000000000000000000000000000000000000000000000003CFEDC
:4230BA00000000000000000000000000000000000000000000000000000000003001000000000000000000000000000000000000000000000000000000000000000000000CFF98
:4230FC00000000000000000000000000000000000000000000000000000000000010000000000000000000000000000000000000000000000000000000000000000000002CFF57
:42313E00000000000000000000000000000000000000000000000000000000003C000000000000000000000000000000000000000000000000000000000000000000000000FE15
:4231800008000000000000000000000000000000000000000000000000000000041100000000000000000000000000000000000000000000000000000000000000000000B9FF38
:4231C200000000000000000000000000000000000000000000000000000000000000000000000000000000000000000000000000000000000000000000000000000000003CFE91
:42320400000000000000000000000000000000000000000000000000000000003C000000000000000000000000000000000000000000000000000000000000000000000000FE4E
:4232460004000000000000000000000000000000000000000000000000000000000000000000000000000000000000000000000000000000000000000000000000000080F4FED0
:42328800000000000000000000000000000000000000000000000000000000003000000000000000000000000000000000000000000000000000000000000000000000000CFECA
:4232CA00000000000000000000000000000000000000000000000000000000000000000000000000000000000000000000000000000000000000000000000000000000001EFCA8
:42330C002000048000100002400008000120000480001000024000080001200004000000000010000240000800012000048000100002400008000120000480001000020034FC1D
:42334E00000000000000000000000000000000000000000000000000000000000000000000000000000000000000000000000000000000000000000000000000000000003CFE03
:4233900024000480001000024000080001200004800010000240000800012000040000000000100002400008000120000480001000024000080001200004800010000280EDFD5B
:4233D2000C00000000000000000000000000000000000000000000000000000020000000000000000000000000000000000000000000000000000000000000000000008054FEBB
:423414002000048000100002400008000120000480001000024000080001200000000000000010000240000800012000048000100002400008000120000480001000020030FC1C
:423456000800000000000000000000000000000000000000000000000000000000000000000000000000000000000000000000000000000000000000000000000000008025FF88
:423498002000048000100002400008000120000480001000024000080001200004000000000010000240000800012000048000100002400008000120000480001000020034FC90
:4234DA00000000000000000000000000000000000000000000000000000000000000000000000000000000000000000000000000000000000000000000000000000000003CFE76
:42351C00000000000000000000000000000000000000000000000000000000000000000000000000000000000000000000000000000000000000000000000000000000003CFE33
:42355E00000000000000000000000000000000000000000000000000000000000000000000000000000000000000000000000000000000000000000000000000000000003CFEF1
:4235A0000000000000000000000000000000000000000000000000000000000040000000000000000000000000000000000000000000000000000000000000000000004038FE33
:4235E200000000000000000000000000000000000000000000000000000000000000000000000000000000000000000000000000000000000000000000000000000000003CFE6D
:42362400000000000000000000000000000000000000000000000000000000000000000000000000000000000000000000000000000000000000000000000000000000003CFE2A
:42366600000000000000000000000000000000000000000000000000000000000000000000000000000000000000000000000000000000000000000000000000000000001EFC08
:4236A800000000000000000000000000000000000000000000000000000000000000000000000000000000000000000000000000000000000000000000000000000000003CFEA6
:4236EA00000000000000000000000000000000000000000000000000000000000000000000000000000000000000000000000000000000000000000000000000000000003CFE64
:42372C0000000000000000000000000000000000000000000000000000000000800000000000000000000000000000000000000000000000000000000000000000000000BCFE21
:42376E00000000000000000000000000000000000000000000000000000000000000000000000000000000000000000000000000000000000000000000000000000000003CFEDF
:4237B0000000000000000000000000000000000000000000000000000000000000000000000000000000000000000000000000000000000000000000000000000000004078FE21
:4237F200000000000000000000000000000000000000000000000000000000000000000000000000000000000000000000000000000000000000000000000000000000003CFE5B
:4238340000000000000000000000000000000000000000000000000000000000000800000000000000000000000000000000000000000000000000000000000000000000B4FE98
:42387600000000000000000000000000000000000000000000000000000000000020000000000000000000000000000000000000000000000000000000000000000000001CFCD8
:4238B800000000000000000000000000000200000000000000000000000002000000000000000000000000000000000000000200000000000000000000000000000000003CFC90
:4238FA000000000000000000000000000008000000000000000000000000040000000000000000000000000000000000000004000000000000000000000000000000000074FE0A
:42393C00000000000000000000000000000000000000000000000000000000000000000000000000000000000000000000000000000000000000000000000000000000003CFE0F
:42397E00000000000000000000000000000000000000000000000000000000000000000000000000000000000000000000000000000000000000000000000000000000003CFECD
:4239C000000000000000000000000000000000000000000000000000000000000000000000000000000000000000000000000000000000000000000000000000000000003CFE8B
:423A0200000000000000000000000000000000000000000000000000000000000000000000000000000000000000000000000000000000000000000000000000000000003CFE48
:423A4400000000000000000000000000000000000000000000000000000000000000000000000000000000000000000000000000000000000000000000000000000000003CFE06
:423A8600000000000000000000000000000000000000000000000000000000000000000000000000000000000000000000000000000000000000000000000000000000003CFEC4
:423AC800000000000000000000000000000000000000000000000000000000000000000000000000000000000000000000000000000000000000000000000000000000003CFE82
:423B0A00000000000000000000000000000000000000000000000000000000000000000000000000000000000000000000000000000000000000000000000000000000003CFE3F
:423B4C00000000000000000000000000000000000000000000000000000000000000000000000000000000000000000000000000000000000000000000000000000000003CFEFD
:423B8E00000000000000000000000000000000000000000000000000000000000000000000000000000000000000000000000000000000000000000000000000000000003CFEBB
:423BD000000000000000000000000000000000000000000000000000000000000000000000000000000000000000000000000000000000000000000000000000000000003CFE79
:423C1200000000000000000000000000000000000000000000000000000000000000000000000000000000000000000000000000000000000000000000000000000000003CFE36
:423C5400000000000000000000000000000000000000000000000000000000000000000000000000000000000000000000000000000000000000000000000000000000003CFEF4
:423C9600000000000000000000000000000000000000000000000000000000000000000000000000000000000000000000000000000000000000000000000000000000003CFEB2
:423CD800000000000000000000000000000000000000000000000000000000000000000000000000000000000000000000000000000000000000000000000000000000003CFE70
:423D1A00000000000000000000000000000000000000000100000000000000002000000000000000000000000000000000000000000000000000000000000000000000000CFF3B
:423D5C00000000000000000000000000000000000000000000000000000000000000000000000000000000000000000000000000000000000000000000000000000000003CFEEB
:423D9E00000000000000000000000000000000000000000000000000000000000000000000000000000000000000000000000000000000000000000000000000000000003CFEA9
:423DE000000000000000000000000000000000000000000000000000000000000000000000000000000000000000000000000000000000000000000000000000000000003CFE67
:423E2200000000000000000000000000000000000000000000000000000000000000000000000000000000000000000000000000000000000000000000000000000000003CFE24
:423E6400000000000000000000000000000000000000000000000000000000000000000000000000000000000000000000000000000000000000000000000000000000003CFEE2
:423EA600000000000000000000000000000000000000000000000000000000000000000000000000000000000000000000000000000000000000000000000000000000003CFEA0
:423EE8000000000000000000000000000000000000000010000000000004020000000000000000000000000000000000000000000000000000000000000000000000000028FC5E
:423F2A0000000000000000000000000000000000000000000000000000010800000000000000000000000000000000000000000000000000000000000000000000000000A4FFA9
:423F6C00000000000000000000000000000000000000002000000000000000000000000000000000000000000000000000000000000000000000000000000000000000001CFED9
:423FAE00000000000000000000000000000000000000000000000000000000000000000000000000000000000000000000000000000000000000000000000000000000003CFE97
:423FF000000000000000000000000000000000000000000000000000000000000000000000000000000000000000000000000000000000000000000000000000000000003CFE55
:42403200000000000000000000000000000000000000000000000000000000000000000000000000000000000000000000000000000000000000000000000000000000003CFE12
:42407400000000000000000000000000000000000000000000000000000000000000000000000000000000000000000000000000000000000000000000000000000000003CFED0
:4240B600000000000000000000000000000000000000000000000000000000000000000000000000000000000000000000000000000000000000000000000000000000003CFE8E
:4240F800000000000000000000000000000000000000000000000000000000000000000000000000000000000000000000000000000000000000000000000000000000003CFE4C
:42413A00000000000000000000000000000000000000000000000000000000000000000000000000000000000000000000000000000000000000000000000000000000003CFE09
:42417C00000000000000000000000000000000000000000000000000000000000000000000000000000000000000000000000000000000000000000000000000000000002DFFD5
:4241BE00000000000000000000000000000000000000000000000000000000000000000000000000000000000000000000000000000000000000000000000000000000003CFE85
:42420000000000000000000000000000000000000000000000000000000000000000000000000000000000000000000000000000000000000000000000000000000000003CFE42
:42424200000000000000000000000000000000000000000000000000000000000000000000000000000000000000000000000000000000000000000000000000000000003CFE00
:42428400000000000000000000000000000000000000000000000000000000000000000000000000000000000000000000000000000000000000000000000000000000003CFEBE
:4242C600000000000000000000000000000000000000000000000000000000000000000000000000000000000000000000000000000000000000000000000000000000003CFE7C
:42430800000000000000000000000000000000000000000000000000000000000000000000000000000000000000000000000000000000000000000000000000000000003CFE39
:42434A00000000000000000000000000000000000000000000000000000000000000000000000000000000000000000000000000000000000000000000000000000000003CFEF7
:42438C00000000000000000000000000000000000000000000000000000000000000000000000000000000000000000000000000000000000000000000000000000000003CFEB5
:4243CE00000000000000000000000000000000000000000000000000000000000000000000000000000000000000000000000000000000000000000000000000000000003CFE73
:42441000000000000000000000000000000000000000000000000000000000000000000000000000000000000000000000000000000000000000000000000000000000003CFE30
:42445200000000000000000000000000000000000000000000000000000000000000000000000000000000000000000000000000000000000000000000000000000000003CFEEE
:42449400000000000000000000000000000000000000000000000000000000000000000000000000000000000000000000000000000000000000000000000000000000003CFEAC
:4244D600000000000000000000000000000000000000000000000000000000000000000000000000000000000000000000000000000000000000000000000000000000001EFC8A
:42451800000000000000000000000000000000000000000000000000000000000000000000000000000000000000000000000000000000000000000000000000000000003CFE27
:42455A00000000000000000000000000000000000000000000000000000000000000000000000000000000000000000000000000000000000000000000000000000000003CFEE5
:42459C000800000000000000000000000000000000000000000000000000000000000000000000000000000000000000000000000000000000000000000000000000008025FF31
:4245DE0000000000000000000000000000000000000000000000000000000000000000000000000000000000000000000000000000000000000000000000000000000080B4FE69
:42462000000000000000000000000000000000000000000000000000000000000000000000000000000000000000000000000000000000000000000000000000000000003CFE1E
:4246620004000000000000000000000000000000000000000000000000000000000000000000000000000000000000000000000000000000000000000000000000000080E5FFAE
:4246A400000000000000000000000000000000000000000000000000000000000000000000000000000000000000000000000000000000000000000000000000000000003CFE9A
:4246E600000000000000000000000000000000000000000000000000000000000000000000000000000000000000000000000000000000000000000000000000000000003CFE58
:42472800000000000000000000000000000000000000000000000000000000000000000000000000000000000000000000000000000000000000000000000000000000003CFE15
:42476A00000000000000000000000000000000000000000000000000000000000000000000000000000000000000000000000000000000000000000000000000000000003CFED3
:4247AC00040000000000000000000000000000000000000000000000000000000000000000000000000000000000000000000000000000000000000000000000000000006DFF5B
:4247EE000C000000000000000000000000000000000000000000000000000000000000000000000000000000000000000000000000000000000000000000000000000000FCFE83
:42483000000000000000000000000000000000000000000000000000000000000000000000000000000000000000000000000000000000000000000000000000000000003CFE0C
:424872000800000000000000000000000000000000000000000000000000000000000000000000000000000000000000000000000000000000000000000000000000008034FE4A
:4248B400000000000000000000000000000000000000000000000000000000000000000000000000000000000000000000000000000000000000000000000000000000003CFE88
:4248F600000000000000000000000000000000000000000000000000000000000000000000000000000000000000000000000000000000000000000000000000000000003CFE46
:42493800000000000000000000000000000000000000000000000000000000000000000000000000000000000000000000000000000000000000000000000000000000003CFE03
:42497A00000000000000000000000000000000000000000000000000000000000000000000000000000000000000000000000000000000000000000000000000000000003CFEC1
:4249BC00040000000000000000000000000000000000000000000000000000000000000000000000000000000000000000000000000000000000000000000000000000006DFF49
:4249FE000C000000000000000000000000000000000000000000000000000000000000000000000000000000000000000000000000000000000000000000000000000000FCFE71
:424A4000000000000000000000000000000000000000000000000000000000000000000000000000000000000000000000000000000000000000000000000000000000003CFEFA
:424A82000800000000000000000000000000000000000000000000000000000000000000000000000000000000000000000000000000000000000000000000000000008034FE38
:424AC400000000000000000000000000000000000000000000000000000000000000000000000000000000000000000000000000000000000000000000000000000000003CFE76
:424B0600000000000000000000000000000000000000000000000000000000000000000000000000000000000000000000000000000000000000000000000000000000001EFC53
:424B4800000000000000000000000000000000000000000000000000000000000000000000000000000000000000000000000000000000000000000000000000000000003CFEF1
:424B8A00000000000000000000000000000000000000000000000000000000000000000000000000000000000000000000000000000000000000000000000000000000003CFEAF
:424BCC0004000000000000000000000000000000000000000000000000000000000000000000000000000000000000000000000000000000000000000000000000000080E5FF3F
:424C0E000C00000000000000000000000000000000000000000000000000000000000000000000000000000000000000000000000000000000000000000000000000008074FE66
:424C5000000000000000000000000000000000000000000000000000000000000000000000000000000000000000000000000000000000000000000000000000000000003CFEE8
:424C92000800000000000000000000000000000000000000000000000000000000000000000000000000000000000000000000000000000000000000000000000000008025FF34
:424CD400000000000000000000000000000000000000000000000000000000000000000000000000000000000000000000000000000000000000000000000000000000003CFE64
:424D1600000000000000000000000000000000000000000000000000000000000000000000000000000000000000000000000000000000000000000000000000000000003CFE21
:424D5800000000000000000000000000000000000000000000000000000000000000000000000000000000000000000000000000000000000000000000000000000000003CFEDF
:424D9A00000000000000000000000000000000000000000000000000000000000000000000000000000000000000000000000000000000000000000000000000000000003CFE9D
:424DDC00040000000000000000000000000000000000000000000000000000000000000000000000000000000000000000000000000000000000000000000000000000006DFF25
:424E1E000C000000000000000000000000000000000000000000000000000000000000000000000000000000000000000000000000000000000000000000000000000000FCFE4C
:424E6000000000000000000000000000000000000000000000000000000000000000000000000000000000000000000000000000000000000000000000000000000000003CFED6
:424EA2000800000000000000000000000000000000000000000000000000000000000000000000000000000000000000000000000000000000000000000000000000008034FE14
:424EE400000000000000000000000000000000000000000000000000000000000000000000000000000000000000000000000000000000000000000000000000000000003CFE52
:424F2600000000000000000000000000000000000000000000000000000000000000000000000000000000000000000000000000000000000000000000000000000000001EFC2F
:424F6800000000000000000000000000000000000000000000000000000000000000000000000000000000000000000000000000000000000000000000000000000000003CFECD
:424FAA00000000000000000000000000000000000000000000000000000000000000000000000000000000000000000000000000000000000000000000000000000000003CFE8B
:424FEC0004000000000000000000000000000000000000000000000000000000000000000000000000000000000000000000000000000000000000000000000000000080E5FF1B
:42502E000C00000000000000000000000000000000000000000000000000000000000000000000000000000000000000000000000000000000000000000000000000008074FE42
:42507000000000000000000000000000000000000000000000000000000000000000000000000000000000000000000000000000000000000000000000000000000000003CFEC4
:4250B2000800000000000000000000000000000000000000000000000000000000000000000000000000000000000000000000000000000000000000000000000000008025FF10
:4250F400000000000000000000000000000000000000000000000000000000000000000000000000000000000000000000000000000000000000000000000000000000003CFE40
:42513600000000000000000000000000000000000000000000000000000000000000000000000000000000000000000000000000000000000000000000000000000000003CFEFD
:42517800000000000000000000000000000000000000000000000000000000000000000000000000000000000000000000000000000000000000000000000000000000003CFEBB
:4251BA00000000000000000000000000000000000000000000000000000000000000000000000000000000000000000000000000000000000000000000000000000000003CFE79
:4251FC00040000000000000000000000000000000000000000000000000000000000000000000000000000000000000000000000000000000000000000000000000000006DFF01
:42523E000C000000000000000000000000000000000000000000000000000000000000000000000000000000000000000000000000000000000000000000000000000000FCFE28
:42528000000000000000000000000000000000000000000000000000000000000000000000000000000000000000000000000000000000000000000000000000000000003CFEB2
:4252C2000800000000000000000000000000000000000000000000000000000000000000000000000000000000000000000000000000000000000000000000000000008034FEF0
:42530400000000000000000000000000000000000000000000000000000000000000000000000000000000000000000000000000000000000000000000000000000000003CFE2D
:42534600000000000000000000000000000000000000000000000000000000000000000000000000000000000000000000000000000000000000000000000000000000001EFC0B
:425388002000048000100002400008000120000480001000024000080001200004000000000010000240000800012000048000100002400008000120000480001000020034FC81
:4253CA00000000000000000000000000000000000000000000000000000000000000000000000000000000000000000000000000000000000000000000000000000000003CFE67
:42540C0024000480001000024000080001200004800010000240000800012000040000000000100002400008000120000480001000024000080001200004800010000280EDFDBE
:42544E000C00000000000000000000000000000000000000000000000000000000000000000000000000000000000000000000000000000000000000000000000000008074FE1E
:425490002000048000100002400008000120000480001000024000080001200004000000000010000240000800012000048000100002400008000120000480001000020034FC78
:4254D2000800000000000000000000000000000000000000000000000000000000000000000000000000000000000000000000000000000000000000000000000000008025FFEC
:425514002000048000100002400008000120000480001000024000080001200004000000000010000240000800012000048000100002400008000120000480001000020034FCF3
:42555600000000000000000000000000000000000000000000000000000000000000000000000000000000000000000000000000000000000000000000000000000000003CFED9
:42559800000000000000000000000000000000000000000000000000000000000000000000000000000000000000000000000000000000000000000000000000000000003CFE97
:4255DA00000000000000000000000000000000000000000000000000000000000000000000000000000000000000000000000000000000000000000000000000000000003CFE55
:42561C00000000000000000000000000000000000000000000000000000000000000000000000000000000000000000000000000000000000000000000000000000000003CFE12
:42565E00000000000000000000000000000000000000000000000000000000000000000000000000000000000000000000000000000000000000000000000000000000003CFED0
:4256A000000000000000000000000000000000000000000000000000000000000000000000000000000000000000000000000000000000000000000000000000000000003CFE8E
:4256E2000000000000000000000000000000000000000000000000000000000000000000000000000000000000000000000000000000000000000000000000000000004078FED0
:42572400000000000000000000000000000000000000000000000000000000000000000000000000000000000000000000000000000000000000000000000000000000003CFE09
:42576600000000000000000000000000000000000000000000000000000000000000000000000000000000000000000000000000000000000000000000000000000000003CFEC7
:4257A800000000000000000000000000000000000000000000000000000000000000000000000000000000000000000000000000000000000000000000000000000000003CFE85
:4257EA00000000000000000000000000000000000000000000000000000000000000000000000000000000000000000000000000000000000000000000000000000000003CFE43
:42582C000000000000000000000000000000000000000000000000000000000000000000000000000000000000000000000000000000000000000000000000000000004078FE84
:42586E00000000000000000000000000000000000000000000000000000000000000000000000000000000000000000000000000000000000000000000000000000000003CFEBE
:4258B000002000000000000000000000000000000000000000000000000000000000000000000000000000000000000000000000000000000000000000000000000000001CFE7C
:4258F200000001000000000000000000000000000000000000000000000000000000000000000000000000000000000000000000000000000000000000000000000000003CFF38
:42593400000000000000000000000000000000000000000000000000000000000000000000000000000000200000000000000000000000000000000000000000000000003CFCD9
:425976000000000000000000000000000000000000000000000000000000000000000000000000000000004000000000000000000000000000000000000000000000000078FE39
:4259B800000000000000000000000000000000000000000000000000000000000000000000000000000000000000000000000000000000000000000000000000000000003CFE73
:4259FA00000000000000000000000000000000000000000000000000000000000000000000000000000000000000000000000000000000000000000000000000000000003CFE31
:425A3C00000000000000000000000000000000000000000000000000000000000000000000000000000000000000000000000000000000000000000000000000000000003CFEEE
:425A7E00000000000000000000000000000000000000000000000000000000000000000000000000000000000000000000000000000000000000000000000000000000003CFEAC
:425AC000000000000000000000000000000000000000000000000000000000000000000000000000000000000000000000000000000000000000000000000000000000003CFE6A
:425B0200000000000000000000000000000000000000000000000000000000000000000000000000000000000000000000000000000000000000000000000000000000001EFC47
:425B4400000000000000000000000000000000000000000000000000000000000000000000000000000000000000000000000000000000000000000000000000000000003CFEE5
:425B8600000000000000000000000000000000000000000000000000000000000000000000000000000000000000000000000000000000000000000000000000000000003CFEA3
:425BC800000000000000000000000000000000000000000000000000000000000000000000000000000000000000000000000000000000000000000000000000000000003CFE61
:425C0A00000000000000000000000000000000000000000000000000000000000000000000000000000000000000000000000000000000000000000000000000000000003CFE1E
:425C4C00000000000000000000000000000000000000000000000000000000000000000000000000000000000000000000000000000000000000000000000000000000003CFEDC
:425C8E00000000000000000000000000000000000000000000000000000000000000000000000000000000000000000000000000000000000000000000000000000000003CFE9A
:425CD000000000000000000000000000000000000000000000000000000000000000000000000000000000000000000000000000000000000000000000000000000000003CFE58
:425D1200000000000000000000000000000000000000000000000000000000000000000000000000000000000000000000000000000000000000000000000000000000003CFE15
:425D5400000000000000000000000000000000000000000000000000000000000000000000000000000000000000000000000000000000000000000000000000000000002DFFE1
:425D9600000000000000000000000000000000000000000000000000000000000000000000000000000000000000000000000000000000000000000000000000000000003CFE91
:425DD800000000000000000000000000000000000000000000000000000000000000000000000000000000000000000000000000000000000000000000000000000000003CFE4F
:425E1A00000000000000000000000000000000000000000000000000000000000000000000000000000000000000000000000000000000000000000000000000000000003CFE0C
:425E5C00000000000000000000000000000000000000000000000000000000000000000000000000000000000000000000000000000000000000000000000000000000003CFECA
:425E9E00000000000000000000000000000000000000000000000000000000000000000000000000000000000000000000000000000000000000000000000000000000003CFE88
:425EE0000000000000000000000000000000000000000000000000000000000000000000000000000000000000000000000000000000000000000000000000000000004078FECA
:425F2200000000000000000000000000000000000000000000000000000000000000000000000000000000000000000000000000000000000000000000000000000000003CFE03
:425F6400000000000000000000000000000000000000000000000000000000002000000000000000000000000000000000000001000000000000000000000000000000001CFFBF
:425FA60000000000000000000000000000000000000000000000000000000000000000000000000000000000000000000000800000000000000000000000000000000000BCFE7F
:425FE8000000000000000000000000000000000000000000000000000000000008000000000000000000000000000000000000000000000000000000000000000000000034FE3D
:42602A00000000000000000000000000000000000000000000000000000000000000000000000000000000000000000000000000000000000000000000000000000000003CFEFA
:42606C00000000000000000000000000000000000000000000000000000000000000000000000000000000000000000000000000000000000000000000000000000000003CFEB8
:4260AE00000000000000000000000000000000000000000000000000000000000000000000000000000000000000000000000000000000000000000000000000000000003CFE76
:4260F000000000000000000000000000000000000000000000000000000000000000000000000000000000000000000000000000000000000000000000000000000000003CFE34
:42613200000000000000000000000000000000000000000000000000000000000000000000000000000000000000000000000000000000000000000000000000000000003CFEF1
:42617400000000000000000000000000000000000000000000000000000000000000000000000000000000000000000000000000000000000000000000000000000000003CFEAF
:4261B6000000000000000000000000000000000000000000000000000000000000000000000000000000000000000000000000000000000000000000000000000000004078FEF1
:4261F800000000000000000000000000000000000000000000000000000000000000000000000000000000000000000000000000000000000000000000000000000000003CFE2B
:42623A00000000000000000000000000000000000000000000000000000000000000000000000000000000000000000000000000000000000000000000000000000000003CFEE8
:42627C00000000000000000000000000000000000000000000000000000000000000000000000000000000000000000000000000000000000000000000000000000000003CFEA6
:4262BE00000000000000000000000000000000000000000000000000000000000000000000000000000000000000000000000000000000000000000000000000000000003CFE64
:42630000000000000000000000000000000000000000000000000000000000000000000000000000000000000000000000000000000000000000000000000000000000003CFE21
:42634200000000000000000000000000000000000000000000000000000000000000000000000000000000000000000000000000000000000000000000000000000000003CFEDF
:42638400000000000000000000000000000000000000000000000000000000000000000000000000000000000000000000000000000000000000000000000000000000003CFE9D
:4263C600000000000000000000000000000000000000000000000000000000000000000000000000000000000000000000000000000000000000000000000000000000003CFE5B
:42640800000000000000000000000000000000000000000000000000000000000000000000000000000000000000000000000000000000000000000000000000000000003CFE18
:42644A00000000000000000000000000000000000000000000000000000000000000000000000000000000000000000000000000000000000000000000000000000000003CFED6
:42648C00000000000000000000000000000000000000000000000000000000000000000000000000000000000000000000000000000000000000000000000000000000003CFE94
:4264CE00000000000000000000000000000000000000000000000000000000000000000000000000000000000000000000000000000000000000000000000000000000003CFE52
:42651000000000000000000000000000000000000000000000000000000000000000000000000000000000000000000000000000000000000000000000000000000000003CFE0F
:42655200000000000000000000000000000000000000000000000000000000000000000000000000000000000000000000000000000000000000000000000000000000001EFCED
:42659400000000000000000000000000000000000000000000000000000000000000000000000000000000000000000000000000000000000000000000000000000000003CFE8B
:4265D600000000000000000000000000000000000000000000000000000000000000000000000000000000000000000000000000000000000000000000000000000000003CFE49
:426618000800000000000000000000000000000000000000000000000000000000000000000000000000000000000000000000000000000000000000000000000000008025FF94
:42665A0000000000000000000000000000000000000000000000000000000000000000000000000000000000000000000000000000000000000000000000000000000080B4FECC
:42669C00000000000000000000000000000000000000000000000000000000000000000000000000000000000000000000000000000000000000000000000000000000003CFE82
:4266DE0004000000000000000000000000000000000000000000000000000000000000000000000000000000000000000000000000000000000000000000000000000080E5FF12
:42672000000000000000000000000000000000000000000000000000000000000000000000000000000000000000000000000000000000000000000000000000000000003CFEFD
:42676200000000000000000000000000000000000000000000000000000000000000000000000000000000000000000000000000000000000000000000000000000000003CFEBB
:4267A400000000000000000000000000000000000000000000000000000000000000000000000000000000000000000000000000000000000000000000000000000000003CFE79
:4267E600000000000000000000000000000000000000000000000000000000000000000000000000000000000000000000000000000000000000000000000000000000003CFE37
:42682800040000000000000000000000000000000000000000000000000000000000000000000000000000000000000000000000000000000000000000000000000000006DFFBE
:42686A000C000000000000000000000000000000000000000000000000000000000000000000000000000000000000000000000000000000000000000000000000000000FCFEE6
:4268AC00000000000000000000000000000000000000000000000000000000000000000000000000000000000000000000000000000000000000000000000000000000003CFE70
:4268EE000800000000000000000000000000000000000000000000000000000000000000000000000000000000000000000000000000000000000000000000000000008034FEAE
:42693000000000000000000000000000000000000000000000000000000000000000000000000000000000000000000000000000000000000000000000000000000000003CFEEB
:42697200000000000000000000000000000000000000000000000000000000000000000000000000000000000000000000000000000000000000000000000000000000001EFCC9
:4269B400000000000000000000000000000000000000000000000000000000000000000000000000000000000000000000000000000000000000000000000000000000003CFE67
:4269F600000000000000000000000000000000000000000000000000000000000000000000000000000000000000000000000000000000000000000000000000000000003CFE25
:426A38000800000000000000000000000000000000000000000000000000000000000000000000000000000000000000000000000000000000000000000000000000008025FF70
:426A7A0000000000000000000000000000000000000000000000000000000000000000000000000000000000000000000000000000000000000000000000000000000080B4FEA8
:426ABC00000000000000000000000000000000000000000000000000000000000000000000000000000000000000000000000000000000000000000000000000000000003CFE5E
:426AFE0004000000000000000000000000000000000000000000000000000000000000000000000000000000000000000000000000000000000000000000000000000080E5FFEE
:426B4000000000000000000000000000000000000000000000000000000000000000000000000000000000000000000000000000000000000000000000000000000000003CFED9
:426B8200000000000000000000000000000000000000000000000000000000000000000000000000000000000000000000000000000000000000000000000000000000001EFCB7
:426BC400000000000000000000000000000000000000000000000000000000000000000000000000000000000000000000000000000000000000000000000000000000003CFE55
:426C0600000000000000000000000000000000000000000000000000000000000000000000000000000000000000000000000000000000000000000000000000000000003CFE12
:426C48000800000000000000000000000000000000000000000000000000000000000000000000000000000000000000000000000000000000000000000000000000008025FF5E
:426C8A0000000000000000000000000000000000000000000000000000000000000000000000000000000000000000000000000000000000000000000000000000000080B4FE96
:426CCC00000000000000000000000000000000000000000000000000000000000000000000000000000000000000000000000000000000000000000000000000000000002DFF5A
:426D0E00040000000000000000000000000000000000000000000000000000000000000000000000000000000000000000000000000000000000000000000000000000004FFDF3
:426D5000000000000000000000000000000000000000000000000000000000000000000000000000000000000000000000000000000000000000000000000000000000003CFEC7
:426D9200100000000000000000000000000000000000000000000000000000000000000000000000000000000000000000000000000000000000000000000000000000001EFD94
:426DD400000000000000000000000000000000000000000000000000000000000000000000000000000000000000000000000000000000000000000000000000000000003CFE43
:426E1600000000000000000000000000000000000000000000000000000000000000000000000000000000000000000000000000000000000000000000000000000000003CFE00
:426E580004000000000000000000000000000000000000000000000000000000000000000000000000000000000000000000000000000000000000000000000000000080E5FF90
:426E9A0004000000000000000000000000000000000000000000000000000000000000000000000000000000000000000000000000000000000000000000000000000080F4FE40
:426EDC00000000000000000000000000000000000000000000000000000000000000000000000000000000000000000000000000000000000000000000000000000000003CFE3A
:426F1E000C00000000000000000000000000000000000000000000000000000000000000000000000000000000000000000000000000000000000000000000000000008065FF41
:426F6000000000000000000000000000000000000000000000000000000000000000000000000000000000000000000000000000000000000000000000000000000000003CFEB5
:426FA200000000000000000000000000000000000000000000000000000000000000000000000000000000000000000000000000000000000000000000000000000000003CFE73
:426FE400000000000000000000000000000000000000000000000000000000000000000000000000000000000000000000000000000000000000000000000000000000003CFE31
:42702600000000000000000000000000000000000000000000000000000000000000000000000000000000000000000000000000000000000000000000000000000000003CFEEE
:4270680004000000000000000000000000000000000000000000000000000000000000000000000000000000000000000000000000000000000000000000000000000080E5FF7E
:4270AA000C00000000000000000000000000000000000000000000000000000000000000000000000000000000000000000000000000000000000000000000000000008074FEA6
:4270EC00000000000000000000000000000000000000000000000000000000000000000000000000000000000000000000000000000000000000000000000000000000003CFE28
:42712E000800000000000000000000000000000000000000000000000000000000000000000000000000000000000000000000000000000000000000000000000000008025FF73
:42717000000000000000000000000000000000000000000000000000000000000000000000000000000000000000000000000000000000000000000000000000000000003CFEA3
:4271B200000000000000000000000000000000000000000000000000000000000000000000000000000000000000000000000000000000000000000000000000000000003CFE61
:4271F400000000000000000000000000000000000000000000000000000000000000000000000000000000000000000000000000000000000000000000000000000000003CFE1F
:42723600000000000000000000000000000000000000000000000000000000000000000000000000000000000000000000000000000000000000000000000000000000003CFEDC
:42727800040000000000000000000000000000000000000000000000000000000000000000000000000000000000000000000000000000000000000000000000000000006DFF64
:4272BA000C000000000000000000000000000000000000000000000000000000000000000000000000000000000000000000000000000000000000000000000000000000FCFE8C
:4272FC00000000000000000000000000000000000000000000000000000000000000000000000000000000000000000000000000000000000000000000000000000000003CFE16
:42733E000800000000000000000000000000000000000000000000000000000000000000000000000000000000000000000000000000000000000000000000000000008034FE53
:42738000000000000000000000000000000000000000000000000000000000000000000000000000000000000000000000000000000000000000000000000000000000003CFE91
:4273C200000000000000000000000000000000000000000000000000000000000000000000000000000000000000000000000000000000000000000000000000000000001EFC6F
:427404002000048000100002400008000120000480001000024000080001200004000000000010000240000800012000048000100002400008000120000480001000020034FCE4
:42744600000000000000000000000000000000000000000000000000000000000000000000000000000000000000000000000000000000000000000000000000000000003CFECA
:42748800280004800010000240000800012000048000100002400008000120000400000000001000024000080001200004800010000240000800012000048000100002802DFDDE
:4274CA0000000000000000000000000000000000000000000000000000000000000000000000000000000000000000000000000000000000000000000000000000000080B4FE4E
:42750C002000048000100002400008000120000480001000024000080001200004000000000010000240000800012000048000100002400008000120000480001000020034FCDB
:42754E0004000000000000000000000000000000000000000000000000000000000000000000000000000000000000000000000000000000000000000000000000000080E5FF93
:427590002000048000100002400008000120000480001000024000080001200004000000000010000240000800012000048000100002400008000120000480001000020034FC57
:4275D200000000000000000000000000000000000000000000000000000000000000000000000000000000000000000000000000000000000000000000000000000000003CFE3D
:42761400000000000000000000000000000000000000000000000000000000000000000000000000000000000000000000000000000000000000000000000000000000003CFEFA
:42765600000000000000000000000000000000000000000000000000000000000000000000000000000000000000000000000000000000000000000000000000000000003CFEB8
:42769800000000000000000000000000000000000000000000000000000000000000000000000000000000000000000000000000000000000000000000000000000000003CFE76
:4276DA000000000000000000000000000000000000000000000000000000000000000000000000000000000000000000000000000000000000000000000000000000004078FEB8
:42771C00000000000000000000000000000000000000000000000000000000000000000000000000000000000000000000000000000000000000000000000000000000003CFEF1
:42775E00000000000000000000000000000000000000000000000000000000000000000000000000000000000000000000000000000000000000000000000000000000001EFCCF
:4277A000000000000000000000000000000000000000000000000000000000000000000000000000000000000000000000000000000000000000000000000000000000003CFE6D
:4277E200000000000000000000000000000000000000000000000000000000000000000000000000000000000000000000000000000000000000000000000000000000003CFE2B
:42782400000000000000000000000000000000000000000000000000000000000000000000000000000000000000000000000000000000000000000000000000000000003CFEE8
:42786600000000000000000000000000000000000000000000000000000000000000000000000000000000000000000000000000000000000000000000000000000000003CFEA6
:4278A8000000000000000000000000000000000000000000000000000000000000000000000000000000000000000000000000000000000000000000000000000000008096FC8C
:4278EA000000000000000000000000000000000000000000000000000000000000000000000000000000000008000000000000000000000000000000000000000000000034FE22
:42792C0000000000000000000000000000000000000000000000000800000000000000000000000000000000000000000000000000000000000000000000000000000000B4FE5F
:42796E000000000000000000000000000000000000000000000000080000000000000000000000000000000020000000000000000000000000000000000000000000000094FE1D
:4279B000000020000000000000000000000000000000000000000000000000000000000000000000000000000000000000000000000000000000000000000000000000001CFC5D
:4279F200000000000000000000000000000000000000000000000000000000000000000000000000000000000000000000000000000000000000000000000000000000003CFE19
:427A3400000020000000000000000000000000000000000000000000000000000000000000000000000000000000000000000000000000000000000000000000000000001CFCD8
:427A7600000000000000000000000000000000000000000000000000000000000000000000000000000000000000000000000000000000000000000000000000000000003CFE94
:427AB800000000000000000000000000000000000000000000000000000000000000000000000000000000000000000000000000000000000000000000000000000000003CFE52
:427AFA00000000000000000000000000000000000000000000000000000000000000000000000000000000000000000000000000000000000000000000000000000000003CFE10
:427B3C00000000000000000000000000000000000000000000000000000000000000000000000000000000000000000000000000000000000000000000000000000000003CFECD
:427B7E00000000000000000000000000000000000000000000000000000000000000000000000000000000000000000000000000000000000000000000000000000000003CFE8B
:427BC000000000000000000000000000000000000000000000000000000000000000000000000000000000000000000000000000000000000000000000000000000000003CFE49
:427C0200000000000000000000000000000000000000000000000000000000000000000000000000000000000000000000000000000000000000000000000000000000003CFE06
:427C4400000000000000000000000000000000000000000000000000000000000000000000000000000000000000000000000000000000000000000000000000000000003CFEC4
:427C860000000000000000000000000000000000000000000000000000000000000000000000000000000000000000000000000000000000000000000000000000000080B4FE8A
:427CC800000000000000000000000000000000000000000000000000000000000000000000000000000000000000000000000000000000000000000000000000000000003CFE40
:427D0A00000000000000000000000000000000000000000000000000000000000000000000000000000000000000000000000000000000000000000000000000000000003CFEFD
:427D4C00000000000000000000000000000000000000000000000000000000000000000000000000000000000000000000000000000000000000000000000000000000003CFEBB
:427D8E00000000000000000000000000000000000000000000000000000000000000000000000000000000000000000000000000000000000000000000000000000000003CFE79
:427DD000000000000000000000000000000000000000000000000000000000000000000000000000000000000000000000000000000000000000000000000000000000003CFE37
:427E1200000000000000000000000000000000000000000000000000000000000000000000000000000000000000000000000000000000000000000000000000000000001EFC14
:427E5400000000000000000000000000000000000000000000000000000000000000000000000000000000000000000000000000000000000000000000000000000000003CFEB2
:427E9600000000000000000000000000000000000000000000000000000000000000000000000000000000000000000000000000000000000000000000000000000000003CFE70
:427ED800000000000000000000000000000000000000000000000000000000000000000000000000000000000000000000000000000000000000000000000000000000003CFE2E
:427F1A000000000000000000000000000000000000000000000000000000000000000000000000000000000000000000000000000000000000000000000000000000004258FE8D
:427F5C00000000000000000000000000000000000000000000000000000000000000000000000000000000000000000000000000000000000000000000000000000000001EFCC9
:427F9E0000000000000000000000000000000060000000000000000000000000000000000000000000000000000000000000000000000000000000000000000000000008F8FC45
:427FE0000000000000000000000000000000000000000000000000000008000000000000000000000000000000000000000000000000000000000000000000000000000034FE25
:42802200000000000000000000000000000000000000000000000000000000000000000000000000000000000000000000000000000000000000000000000000000000003CFEE2
:42806400000000000000000000000000000000000000000000000000000100000000000000000000000000000000000000000000000000000000000000000000000000002CFFAE
:4280A600000000000000000000000000000000000000000000000000000000000000000000000000000000000000000000000000000000000000000000000000000000003CFE5E
:4280E8000200000000000000000000000000000000000000000000000000000000000000000000000000000000000000000000000000000000000000000000000000004058FEBE
:42812A000200000000000000000000000000000000000000000000000000000000000000000000000000000000000000000000000000000000000000000000000000004058FE7B
:42816C00000000000000000000000000000000000000000000000000000000000000000000000000000000000000000000000000000000000000000000000000000000003CFE97
:4281AE00000000000000000000000000000000000000000000000000000000000000000000000000000000000000000000000000000000000000000000000000000000003CFE55
:4281F000000000000000000000000000000000000000000000000000000000000000000000000000000000000000000000000000000000000000000000000000000000003CFE13
:42823200000000000000000000000000000000000000000000000000000000000000000000000000000000000000000000000000000000000000000000000000000000003CFED0
:42827400000000000000000000000000000000000000000000000000000000000000000000000000000000000000000000000000000000000000000000000000000000003CFE8E
:4282B600000000000000000000000000000000000000000000000000000000000000000000000000000000000000000000000000000000000000000000000000000000003CFE4C
:4282F800000000000000000000000000000000000000000000000000000000000000000000000000000000000000000000000000000000000000000000000000000000003CFE0A
:42833A00000000000000000000000000000000000000000000000000000000000000000000000000000000000000000000000000000000000000000000000000000000003CFEC7
:42837C00000000000000000000000000000000000000000000000000000000000000000000000000000000000000000000000000000000000000000000000000000000003CFE85
:4283BE0000000040000000000000000000000000000000000000000000000000000000000000000000002001000000000000260000000000000000000000000000880000C4FEAC
:428400000000000000000000000000000000000000000000000000000000000000000000000000000000000000000000000000040000000000000000000000000000000078FEC0
:4284420000003C08000000000000000000000000000000000000000000000000000000000000000000C000000000000000800700000000000000000000000000F0200000D0FD90
:42848400000034010000000000000000000000000000000000000000000000000000000000000000004000000000000000801004000000000000000000000000D008000000FCD9
:4284C60000000041000000000000000000000000000000000000000000000000000000000000000000008B00000000000000000000000000000000000000000000000100E8FCC3
:4285080000003C00000000000000000000000000000000000000000000000000000000000000000000C003000000000000800700000000000000000000000000F000000070FE4D
:42854A00000000000000000000000000000000000000000000000000000000000000000000000000000003000000000000000000000000000000000000000000004000007CFD33
:42858C00000030040000000000000000000000000000000000000000000000000000000000000000000003000000000000000600000000000000000000000000C0040000A0FC10
:4285CE00000000000000000000000000000000000000000000000000000000000000000000000000000020010000000000002600000000000000000000000000C0040000E2FC82
:4286100000000000000000000000000000000000000000000000000000000000000000000000000000000000000000000000000400000000000000000000000000800000F8FEAE
:4286520000000000000000000000000000000000000000000000000000000000000000000000000000C000000000000000800704000000000000000000000000F040000088FEE5
:42869400080000000000000000000000000000000000000000000000000000000000000000000000004000000000000000804000000000000000000000000000100200808DFC81
:4286D6000000000000000000000000000000000000000000000000000000000000000000000000000000A3000000000000000000000000000000000000000000000000809CFFA4
:4287180000000000000000000000000000000000000000000000000000000000000000000000000000C003000000000000800700000000000000000000000000F00000009DFC4C
:42875A00040000000000000000000000000000000000000000000000000000000000000000000000000003000000000000000000000000000000000000000000000000004FFE89
:42879C00000000000000000000000000000000000000000000000000000000000000000000000000000003000000000000000600000000000000000000000000C0000000D4FFFF
:4287DE00000000000000000000000000000000000000000000000000000000000000000000000000000020010000000000004602000000000000000000000000C0040000A0FC90
:4288200000000000000000000000000000000000000000000000000000000000000000000000000000000000000000000000000000000000000000000000000000800000BCFEDC
:4288620000000000000000000000000000000000000000000000000000000000000000000000000000C000000000000000800700000000000000000000000000F00000008CFE13
:4288A40004000000000000000000000000000000000000000000000000000000000000000000000000400000000000000080100200000000000000000000000010100000A5FCFB
:4288E6000C000000000000000000000000000000000000000000000000000000000000000000000000008300000000000000000000000000000000000000000000000000F4FDD0
:4289280000000000000000000000000000000000000000000000000000000000000000000000000000C003000000000000800700000000000000000000000000F00000008CFD4A
:42896A000800000000000000000000000000000000000000000000000000000000000000000000000000030000000000000000000000000000000000000000000000008034FD0F
:4289AC00000000000000000000000000000000000000000000000000000000000000000000000000000003000000000000000600000000000000000000000000C0000000D4FFED
:4289EE000000004000000000000301000000000000000000000000000000000000000000000000000000130000000000000040020000000000000000000000000048000062FD07
:428A3000000000000000000000000000000000000000000000000000000000000000000000000000000000020000000000000000000000000000000000000000000000001CFEE8
:428A720000003C0800000000C003000000000000000000000000000000000000000000000000000000C0030000000000008001000000000000000000000000003000000024FC27
:428AB40008003400000000004050000000000000000000000000000000000000000000000000000000401002000000000080000000000000000000000000000010000080E9FD6C
:428AF600000000410000000000000000000000000000000000000000000000000000000000000000000000000000000000000600000000000000000000000000C008008000FCB3
:428B380000003C0000000000C003000000000000000000000000000000000000000000000000000000C003000000000000800701000000000000000000000000F02000006CFF36
:428B7A00040000200000000000000000000000000000000000000000000000000000000000000000000000000000000000000600000000000000000000000000C00000800DFF43
:428BBC00000030000000000000030000000000000000000000000000000000000000000000000000000003000000000000000600000000000000000000000000C0000000D4FCAB
:428BFE000000300100000000000000000C8485000000000000000000000000000000000000000000000020010000000000004004000000000000000000000000C048000086FC00
:428C4000000000200000000000000000000000000000000000000000000000000000000000000000000000000000000000000000000000000000000000000000000000003CFC9A
:428C820000003C0000000000000000000FE00100000000000000000000000000000000000000000000C000000000000000800700000000000000000000000000F0800000E0FCF1
:428CC400040004040000000000000000012400010000000000000000000000000000000000000000004000000000000000801601000000000000000000000000100400803DFD97
:428D06000C000000000000000000000000000000000000000000000000000000000000000000000000001300000000000000000800000000000000000000000000000080ECFC9C
:428D480000003C0000000000000000000FE00100000000000000000000000000000000000000000000C083000000000000800700000000000000000000000000F000000079FE8C
:428D8A00080000000000000000000000000000000000000000000000000000000000000000000000000003000000000000000002000000000000000000000000000000008FFC0F
:428DCC000000300000000000000000000C8001000000000000000000000000000000000000000000000003000000000000001600000000000000000000000000C0000000B4FD1E
:428E0E000000001200000000000000000000000000000000000000000000000000000000000000000000130000000000000040020000000000000000000000000048000026FD50
:428E5000000000000000000000000000000000000000000000000000000000000000000000000000000000020000000000000000000000000000000000000000000000001CFEC4
:428E920000000C00000000000000000000000000000000000000000000000000000000000000000000C00301000000000080010000000000000000000000000030000000B8FF66
:428ED4000800040000000000000000000000000000000000000000000000000000000000000000000040080000000000008000000000000000000000000000001000008021FED9
:428F1600000030090000000000000000000000000000000000000000000000000000000000000000000000000000000000004600000000000000000000000000C00200809CFDBF
:428F580000003C00000000000000000000000000000000000000000000000000000000000000000000C003000000000000800701000000000000000000000000F020000041FE01
:428F9A00040030000000000000000000000000000000000000000000000000000000000000000000000000000000000000000600000000000000000000000000C000000097FC08
:428FDC00000030000000000000000000000000000000000000000000000000000000000000000000000003000000000000000600000000000000000000000000C0000000E4FC7A
:42901E008001301200000000000000000000000000000000580800000000000000000000000000000000130000000000000046020000000000000000000000000088000076FC98
:42906000000001000000000000000000000000000000000000000000000000000000000000000000000000020000000000000000000000000000000000000000000000001CFFB0
:4290A200E0813C20000000000000000000000000000000001E08000000000000000000000000000000C003020000000000800704000000000000000000000000F020000034FC19
:4290E400241004020000000000000000000000000000000002000000000000000000000000000000004010000000000000804000000000000000000000000000D0040080C1FFEA
:429126000C00000000000000000000000000000000000000000000000000000000000000000000000000000000000000000000000000000000000000000000000000018074FF07
:42916800E0013C00000000000000000000000000000000001E00000000000000000000000000000000C003000000000000800700000000000000000000000000F000000061FFF0
:4291AA0008000000000000000000000000000000000000000000000000000000000000000000000000000000000000000000000000000000000000000000000000400000CFFD6F
:4291EC00800130000000000000000000000000000000000018000000000000000000000000000000000003000000000000000600000000000000000000000000C0020000C4FEEB
:42922E008001301200000000000301000C8485000000000058080000000000000000000000000000000013000000000000004004000000000000000000000000C048000010FE55
:42927000000001000000000000000000000000000000000000000000000000000000000000000000000000020000000000000000000000000000000000000000000000001CFF9E
:4292B200E0013C1000000000C00301000FE88100000000001E00000000000000000000000000000000C003000000000000800701000000000000000000000000F00000004CFE6E
:4292F4002400850000000000400000008120100000000000020800000000000000000000000000000040200400000000008006000000000000000000000000001010000091FEFB
:429336000C00000000000000000000000000000000000000000000000000000000000000000000000000000000000000000000080000000000000000000000000000000074FE6F
:42937800E0013C0000000000C00300000FE00100000000001E00000000000000000000000000000000C003000000000000800700000000000000000000000000F00000005CFF30
:4293BA000800000000000000000000000000000000000000000000000000000000000000000000000000000000000000000000000000000000000000000000000000008034FEB7
:4293FC008001300000000000000300000C8001000000000018000000000000000000000000000000000003000000000000001604000000000000000000000000C0000000C0FD3C
:42943E00000000000000000000000000000000000000000000000000000000000000000000000000000000000000000000000000000000000000000000000000000000001EFCD2
:429480002000048000100002400008000120000480001000024000080001200004000000000010000240000800012000048000100002400008000120000480001000020034FC48
:4294C200000000000000000000000000000000000000000000000000000000000000000000000000000000000000000000000000000000000000000000000000000000003CFE2E
:42950400280004800010000240000800012000048000100002400008000120000400000000001000024000080001200004800010000240000800012000048000100002802DFD41
:4295460000012000000000000002000008000100000000001000000000000000000000000000000000000200000000000000040000000000000000000000000080000080B8FFEA
:42958800000000800010000200000800000000048000100000400008000120000400000000001000020000080001200004000010000240000800012000048000000002009DFC2D
:4295CA00040000000000000000000000000000000000000000000000000000000000000000000000000000000000000000000000000000000000000000000000000000004FFD0F
:42960C002000048000100002400008000120000480001000024000080001200004000000000010000240000800012000048000100002400008000120000480001000020034FCBA
:42964E00000000000000000000000000000000000000000000000000000000000000000000000000000000000000000000000000000000000000000000000000000000003CFEA0
:42969000000000000000000000000000000000000000000000000000000000000000000000000000000000000000000000000000000000000000000000000000000000003CFE5E
:4296D200000010000000000000000000000000000000000000000000000000000000000000000000000000000000000000000000000000000000000000000000000000002CFF1B
:429714000000800000000000000000000000000000000000000000000000000000000000000000000000000000000000000000000000000000000000000000000000004070FEE5
:42975600000000000000000000000000000000000000000000000000000000000000000000000000000000000000000000000000000000000000000000000000100000003CFF86
:42979800000000000000000000000000000000000000000000000000000000000000000000000000000000010000000000008000000000000000000000000000000000008EFC84
:4297DA00000000000000000000000000000000000000000000000000000000000000000000000000000001000000000000000200000000000000000000000000000000001CFD31
:42981C00000000000000000000000000000000000000000000000000000000000000000000000000000000000000000000000000000000000000000000000000000000003CFED0
:42985E00000000000000000000000000000000000000000000000000000000000000000000000000000000000000000000000000000000000000000000000000000000003CFE8E
:4298A00000000000000000000000000000000000000000000000000000000000000000000000000000000000000000000000000000000000000000000000000000000080B4FE54
:4298E2000000000000000000000000000000000000000000000000000000000000000000000000000000080000000000000000040000000000000000000000002080000070FC2C
:42992400000008400000000000000000000000000000000000000000000000000000000000000000008000000000000000000100000000000000000000000000200000C08EFFCB
:42996600000000000000000000000000000000000000000000000000200000000000000000000000000001000000000000000000000000000000000000000000000000003CFD65
:4299A800000020080000000000000000000000000000000000000000000000000000000000000000000000000000000000000000000000000000000000000000000000009CFCBD
:4299EA00000004200000000000000000000000000000000000000000200000000000000000000000008000000A0000000000000000000000000000000000000000005000C4FD5C
:429A2C0000010800008000320002000800022000048080001000016000000100000000000000000000000090020000000000010000000000000000000000000000006800A0FE02
:429A6E000000000000000000000000000008000000000000000002400000000000000000000000000000000000000000000000000000000000000000000000000000080098FCD0
:429AB00000010000008000100002004000000001200084001000001000000400000000000000000000000000000000000000000000000000000000000000000000000000ACFF2D
:429AF200000000000000000000000000000000000000000000000000000000000000000000000000000000000000000000000000000000000000000000000000000000003CFEF8
:429B3400000000000000000000000000000000000000000000000000000000000000000000000000000000000000000000000001000000000000000000000000000000003CFFB3
:429B76000000000000000000800000000200000000000000000000000000000000000000000000000000000000000000000000000000000000000000000000000000000014FE19
:429BB80000800004000000000000000000000000000000000000000000000000000000000000000000000000000000000000000000000000000000000000000000000000FCFEED
:429BFA000000040000000000000000000000000000000000000000000000000000000000000000000000000000000000000000000000000000000000000000000002000058FCCF
:429C3C000000000000000000000000000000000000000000000000000000000000000000000000000000000400000000000004000000000000000000000000000000000078FE68
:429C7E000000000000000000000000000000000000000000000000000000000000000000000000000000000000000000000000000000000000000000000000004000000078FEEE
:429CC000000000000000000000000000000000000000000000000000000000000000000000000000000000000000000000000000000000000000000000000000000000003CFE28
:429D0200000000000000000000000000000000000000000000000000000000000000000000000000000000000000000000000000000000000000000000000000000000003CFEE5
:429D4400000000000000000000000000000000000000000000000000000000000000000000000000000000000000000000000000000000000000000000000000000000003CFEA3
:429D8600000000000000000000000000000000000000000000000000000000000000000000000000000000000000000000000000000000000000000000000000000000003CFE61
:429DC8000000000000000000400000000000000000000000000000000000000000000000000000000000000000000000000000000000000000000000000000000000000038FEE3
:429E0A000080000000000000000000001000800000000000200000000000000000000000000000000000000000000000000000000000000000000000000000000000000094FD55
:429E4C008000000000000000800000000080000000000000040000000000000000000000000000000000000000000000000000000000000000000000000000000000000069FFE8
:429E8E00000000000000000000000000000000000000000000000000000000000000000000000000000000000000000000000000000000000000000000000000000000001EFC78
:429ED000000000000000000000000000000000000000000000000000000000000000000000000000000000000000000000000000000000000000000000000000000000003CFE16
:429F12000000000000000000000000000000000000000000000000000000000000000000000000000000000000000000000000000000000000000000000000000000004078FE57
:429F5400000000000000000000000000000000000000000000000000000000000000000000000000000000000000000000000000000000000000000000000000000000003CFE91
:429F960000000000000000000000000000000008000000000000000040002000000000000000000000000000000000000000000100000000000000000000000000000040BEFF23
:429FD800000000000000000000000000000000000000000000000000000020000000000000000000000000000000000000000000000000000000000000000000000000003EFEEB
:42A01A0080001000000000000000000A80010008000000000800010020006000000000000000000000005000000000000000000200000000000000000000000000008002B4FED2
:42A05C0000008010000000004000000202400048000000000000080000000100000000000000000000000000000000000000020200000000000000000000000000008005E4FCF4
:42A09E00000000000000000000000000000000000000000000000000000000000000000000000000000000000000000000000200000000000000000000000000000000045CFC22
:42A0E00000000000000000000000000000000000000000000000000000000800000000000000000000000000000000000000000000000000000000000000000000000000B4FE84
:42A12200100000000000000000000000000000000000000000000000000000000000000000000000000000000000000000000000000000000000000000000000000000001EFDD0
:42A16400000000000000000000000000000000000000000000000000000000000000000000000000000000000000000000000000000000000000000000000000000000003CFE7F
:42A1A600000000000000000000000000000000000000000000000000000000000000000000000000000000000000000000000000000000000000000000000000000000003CFE3D
:42A1E80004000000000000000000000000000000000000000000000000000000000000000000000000000000000000000000000000000000000000000000000000000080F4FEBF
:42A22A00040000000000000000000000000000000000000000000000000000000000000000000000000000000000000000000000000000000000000000000000000000400BFDA6
:42A26C00000000000000000000000000000000000000000000000000000000000000000000000000000000000000000000000000000000000000000000000000000000003CFE76
:42A2AE000000000800000000000000000000000000000000000000000000000000000000000000000000800000000000000000010000000000000000000000000020000094FF32
:42A2F000000000000000000000000000000000000000000000000000000000000000000000000000000000000000000000001000000000000000000000000000000200000CFC12
:42A332000000002000000000000000000080000000000000080000000000000000000000000000000000000000000000000000000000000000000000000000000000000034FC11
:42A37400000000000000000000000000000100000000000000000000000000000000000000000000000000000000000000000000000000000000000000000000000000002CFF7B
:42A3B600000000000000000000000000000000000000000000000000000000000000000000000000000000000000000000000000000000000000000000000000000000003CFE2B
:42A3F800000000000000000000000000000000000000000000000000000000000000000000000000000000000000000000000000000000000000000000000000000000003CFEE9
:42A43A00000000000000000000000000000000000000000000000008008C00500000000000000000000000000000000000000000000000000000000000000000000000007CFF81
:42A47C00000000000000000000000000000000000000000000000000000C020000000000000000000000000000000000000000000000000000000000000000000000000030FC64
:42A4BE000000000000000000000000000000000000000000000000000003E04100000000000000000000000000000000000000000000000000000000000000000000000074FFC5
:42A500000000000000000000000000000000000000000000000000000001A00500000000000000000000000000000000000000000000000000000000000000000000000054FD22
:42A542000000000000000000000000000000000000000000000000000C00040002000000000000000000000000000000000000000000000000000000000000000000000098FC31
:42A584000000000000000000000000000000000000000000000000180003E001000000000000000000000000000000000000000000000000000000000000000000000000A8FEF3
:42A5C6000000000000000000000000000000000000000000000000600000008000000000000000000000000000000000000000000000000000000000000000000000000090FCE7
:42A608000000000000000000000000000000000000000000000000601000810500000000000000000000000000000000000000000000000000000000000000000000000040FCDE
:42A64A00000000000000000000000000000000000000000000000060240124000000000000000000000000000000000000000000000000000000000000000000000000000EFF18
:42A68C000000000000000000000000000000000000000000000000600000000000000000000000000000000000000000000000000000000000000000000000000000000018FC18
:42A6CE0000000000000000000000000000000000000000000000007800006000000000000000000000000000000000000000000000000000000000000000000000000000A4FFCF
:42A7100008000000000000000000000000000000000000000000006800002100000000000000000000000000000000000000000000000000000000000000000000000080A9FE4F
:42A7520000000000000000000000000000000000000000000000006000288011010000000000000000000000000000000000000000000000000000000000000000000080B0FC7F
:42A794000000000000000000000000000000000000000000000000780003E2010000000000000000000000000000000000000000000000000000000000000000000000009DFF89
:42A7D600040000000000000000000000000000000000000000000060000C82010000000000000000000000000000000000000000000000000000000000000000000000007FFDD2
:42A81800000000000000000000000000000000000000000000000060008C80010000000000000000000000000000000000000000000000000000000000000000000000008CFC09
:42A85A000000000000000000000000000000000000000000000000680041005000000000000000000000000000000000000000000000000000000000000000000000000084FC43
:42A89C000000000000000000000000000000000000000000000000000004020000000000000000000000000000000000000000000000000000000000000000000000000038FC40
:42A8DE000000000000000000000000000000000000000000000000781000E041000000000000000000000000000000000000000000000000000000000000000000000000F8FE99
:42A920000400000000000000000000000000000000000000000000680020A4090000000000000000000000000000000000000000000000000000000000000000000000001DFFA0
:42A962000C00000000000000000000000000000000000000000000600240080002000000000000000000000000000000000000000000000000000000000000000000000010FEED
:42A9A4000000000000000000000000000000000000000000000000781003E0010000000000000000000000000000000000000000000000000000000000000000000000008CFD7C
:42A9E6000800000000000000000000000000000000000000000000601000000000000000000000000000000000000000000000000000000000000000000000000000008010FD2A
:42AA28000000000000000000000000000000000000000000000000600140842900000000000000000000000000000000000000000000000000000000000000000000000094FE0C
:42AA6A00000000000000000000000000000000000016020000000008000180090000000000000000000000000000000000000000000000000000000000000000000000006AFE98
:42AAAC00000000000000000000000000000000000000000000000000000C0080000000000000000000000000000000000000000000000000000000000000000000000000B8FE26
:42AAEE000000000000000000000000000000000080070000000000180003E0010000000000000000000000000000000000000000000000000000000000000000000000006CFD3A
:42AB3000080000000000000000000000000000008000020000000008000121200000000000000000000000000000000000000000000000000000000000000000000000803DFF53
:42AB72000000000000000000000000000000000000000000000000600C4C02000000000000000000000000000000000000000000000000000000000000000000000000801CFE4D
:42ABB400000000000000000000000000000000008007000000000078000FE00100000000000000000000000000000000000000000000000000000000000000000000000055FE1D
:42ABF600040000000000000000000000000000000000000000000060000C040000000000000000000000000000000000000000000000000000000000000000000000000023FF87
:42AC3800000000000000000000000000000000000006000000000060004C800100000000000000000000000000000000000000000000000000000000000000000000000008FEA1
:42AC7A0000000000060200000000000000000000001602000000000800010010010000000000000000000000000000000000000000000000000000000000000000000000E4FC7E
:42ACBC00000000000000000000000000000000000000000000000000000000000000000000000000000000000000000000000000000000000000000000000000000000003CFE1C
:42ACFE000000008007000000000000000000000080070200000000000003600000000000000000000000000000000000000000000000000000000000000000000000000070FF32
:42AD40000800008000020000000000000000000080000000000000000001200000000000000000000000000000000000000000000000000000000000000000000000000095FE13
:42AD8200000000000000000000000000000000000000000000000000110C8409000000000000000000000000000000000000000000000000000000000000000000000000FCFFEA
:42ADC400000000800700000000000000000000008007000000000018000FE04100000000000000000000000000000000000000000000000000000000000000000000000098FE61
:42AE060004000000000000000000000000000000000000000000006000008001000000000000000000000000000000000000000000000000000000000000000000000080C8FCE1
:42AE48000000000006000000000000000000000000060000000000601000810100000000000000000000000000000000000000000000000000000000000000000000000060FC6E
:42AE8A0000000000000000000000000000000000000000000000000800018011010000000000000000000000000000000000000000000000000000000000000000000000ACFF40
:42AECC00000000000000000000000000000000000000000000000000000000000000000000000000000000000000000000000000000000000000000000000000000000003CFE0A
:42AF0E000000000000000000000000000000000000000000000000180000E08100000000000000000000000000000000000000000000000000000000000000000000000010FD7B
:42AF500004000000000000000000000000000000000000000000000800002000000000000000000000000000000000000000000000000000000000000000000000000000C5FDD1
:42AF92000C0000000000000000000000000000000000000000000060140C0400000000000000000000000000000000000000000000000000000000000000000000000000D0FD20
:42AFD400000000000000000000000000000000000000000000000078000FE00100000000000000000000000000000000000000000000000000000000000000000000000080FC57
:42B016000800000000000000000000000000000000000000000000600000000000000000000000000000000000000000000000000000000000000000000000000000008010FC04
:42B058000000000000000000000000000000000000000000000000600000810100000000000000000000000000000000000000000000000000000000000000000000000000FDD7
:42B09A000000000000000000000000000000000000000000000000080001200000000000000000000000000000000000000000000000000000000000000000000000000084FDCA
:42B0DC00000000000000000000000000000000000000000000000000000000000000000000000000000000000000000000000000000000000000000000000000000000003CFEF8
:42B11E00000000000000000000000000000000000000000000000018000380010000000000000000000000000000000000000000000000000000000000000000000000008CFCCB
:42B160000C000000000000000000000000000000000000000000000800018001000000000000000000000000000000000000000000000000000000000000000000000080E5FEB4
:42B1A200040000000000000000000000000000000000000000000060022C8001020000000000000000000000000000000000000000000000000000000000000000000080E4FEF4
:42B1E400000000000000000000000000000000000000000000000078100FE401000000000000000000000000000000000000000000000000000000000000000000000000C4FDEC
:42B226000C0000000000000000000000000000000000000000000060000C800101000000000000000000000000000000000000000000000000000000000000000000008045FC2B
:42B26800000000000000000000000000000000000000000000000060000C80010000000000000000000000000000000000000000000000000000000000000000000000000CFCAF
:42B2AA000000000006020000000000000000000000160200000000601201801101000000000000000000000000000000000000000000000000000000000000000000000070FFCE
:42B2EC00000000000000000000000000000000000000000000000000000000000000000000000000000000000000000000000000000000000000000000000000000000003CFEE6
:42B32E00000000800700000000000000000000008007000000000078400FE001000000000000000000000000000000000000000000000000000000000000000000000000BCFC6F
:42B37000080000802002000000000000000000008020020000000008044122200000000000000000000000000000000000000000000000000000000000000000000000003DFC87
:42B3B200000000000000000000000000000000000000000000000000000000000000000000000000000000000000000000000000000000000000000000000000000000003CFE1F
:42B3F400000000800700000000000000000000008007000000000078000FE401000000000000000000000000000000000000000000000000000000000000000000000000BCFCE5
:42B4360004000000000000000000000000000000000000000000000000000200000000000000000000000000000000000000000000000000000000000000000000000080F4FC5E
:42B47800000000000600000000000000000000000006000000000060000C80010000000000000000000000000000000000000000000000000000000000000000000000006CFC31
:42B4BA00000000000000000000000000000000000000000000000000000000000000000000000000000000000000000000000000000000000000000000000000000000001EFC36
:42B4FC002000048000100002400008000120000480001000024000080001200004000000000010000240000800012000048000100002400008000120000480001000020034FCAC
:42B53E00000000000000000000000000000000000000000000000000000000000000000000000000000000000000000000000000000000000000000000000000000000003CFE91
:42B580002C0004800010000240000800012000048000100002400008000120000400000000001000024000080001200004800010000240000800012000048000100002806DFD61
:42B5C20004000000040000000000000000000000000400000000004000080001000000000000000000000000000000000000000000000000000000000000000000000080A8FECC
:42B604002000040000100002400008000120000400001000024000000000000004000000000010000240000800012000048000100002400008000120000480001000020084FF78
:42B646000C00000000000000000000000000000000000000000000000000000000000000000000000000000000000000000000000000000000000000000000000000008065FFD2
:42B688002000048000100002400008000120000480001000024000080001200004000000000010000240000800012000048000100002400008000120000480001000020034FC1E
:42B6CA00000000000000000000000000000000000000000000000000000000000000000000000000000000000000000000000000000000000000000000000000000000003CFE04
:42B70C00000000000000000000000000000000000000000000000000000000000000000000000000000000000000000000000000000000000000000000000000000000003CFEC1
:42B74E000000000000000000000000000000000000000000000000000000800000000000000000000000000000000000000000000000000000000000000000000000000034FE07
:42B79000000000000000000000000000000000000000000000000000000000000000000000000000000000000000000000000000000000000000000000000000000000003CFE3D
:42B7D200000000000000000000000000000000000000000000000000000000000000000000000000000000000000000000000000000000000000000000000000000000003CFEFB
:42B81400000000000000000000000000000000000000000000000000000000000000000000000000000000000000000000000000000000000000000000000000000000003CFEB8
:42B85600000000000000000000000000000000000000000000000000000100000000000000000000000000000000000000000000000000000000000000000000000000002CFF84
:42B89800000000000000000000000000000000000000000000000000000000000000000000000000000000000000000000000000000000000000000000000000000000003CFE34
:42B8DA00000000000000000000000000000000000000000000000000000000000000000000000000000000000000000000000000000000000000000000000000000000003CFEF2
:42B91C00000000000000000000000000000000000000000000000000000020040000000000000000000000000000000000000000000000000000000000000000000000005CFC6D
:42B95E00000000000000000000000000000000000000000000000000000000000000000000000000000000000000000000000000000000000000000000000000000000003CFE6D
:42B9A00000000000000000000000000000000000000000000000001000000000000000000000000000000000000000000000000000000000000000000000000000000080A4FF32
:42B9E200000000000000000000000000000000000000000000000000100000000000000000000000000000000000000000000000000000000000000000000000000000003CFFD8
:42BA24000000000000000000000000000000000000000000000000000000804000000000000000000000000000000000000000000000000000000000000000000000000070FEB2
:42BA66000000000000000000000000000000000000000000000000403100200001000000000000000000000000000000000000000000000000000000000000000000000018FEF6
:42BAA8000000000002400000000000000000000000030100000000300000074000000000000000000000020000000000000000000000000000000000000000000000000038FD68
:42BAEA000000000004800000000000000000000000040400000000200000024000000000000000000000000000000000000000000000000000000000000000000000000050FEDE
:42BB2C00000000000000000000000000000000000000000000000000000002000000000000000000000002000000000000000000000000000000000000000000000000003CFE99
:42BB6E00000000000000000000000000000000000000000000000000000000000000000000000000000000000000000000000000000000000000000000000000000000003CFE5B
:42BBB000000000000000000000000000000000000000000000000000000000000000000000000000000000000000000000000000000000000000000000000000000000003CFE19
:42BBF200000000000100000000000000000000000000000000000000000000000100000000000000000000000000000000000000000000000000000000000000000000003CFED5
:42BC340000000000000000000000000000000000000000000000000000004100000000000000000000000000000000000000000000000000000000000000000000000080B0FF5E
:42BC7600000000000000000000000000000000000000000000000000000000000000000000000000000000000000000000000000000000000000000000000000000000003CFE52
:42BCB800000000000000000000000000000000000000000000000000000000000000000000000000000000000000000000000000000000000000000000000000000000003CFE10
:42BCFA00000000000000000000000000000000000000000000000000000000000000000000000000000000000000000000000000000000000000000000000000000000003CFECE
:42BD3C000000000000000000000000000000000000000000000000000008000000000000000000000000000000000000000000000000000000000000000000000000000016FCAB
:42BD7E00000000000000000000000000000000000000000000000000000020000000000000000000000000000000000000000000000000000000000000000000000000001CFC4B
:42BDC000000000000000000000000000000000000000000000000000000000000000000000000000000000000000000000000000000000000000000000000000000000003CFE07
:42BE0200000000000000000000000000000000000000000000000000000000000000000000000000000000000000000000000000000000000000000000000000000000003CFEC4
:42BE4400000000000000000000000000000000000000000000000000000000000000000000000000000000000000000000000000000000000000000000000000000000003CFE82
:42BE860000000000080000000000000000000000000800000000000000000000000000000000000000000000000000000000000000000000000000000000000000000000BCFEB0
:42BEC80000000000080000000000000000000000000800000000000000000000000000000000000000000000000000000000000000000000000000000000000000000000BCFE6E
:42BF0A00000000000000000000000000000000000000000000000000000200010000000000000000000000000000000000000000000000000000000000000000000000000CFCEA
:42BF4C00000000000000000000000000000000000001000000000000000000000000000000000000000000000000000000000000000000000000000000000000000000003CFF77
:42BF8E00000000000000000000000000000000000000000000000000000000000000000000000000000000000000000000000000000000000000000000000000000000003CFE37
:42BFD000000000000000000000000000000000000000000000000000000000000000000000000000000000000000000000000000000000000000000000000000000000003CFEF5
:42C012000000001000000000000000000001000800000000000000001004000000000000000000000000000000000000000000000000000000000000000000000000008002FD40
:42C05400000000000000000000000000000000000000000000000000000000000000000000000000000000000000000000000000000000000000000000000000000000003CFE70
:42C096000000001000000000000000000004000800000000000000002A02000500000000000000000000000000000000000000000000000000000000000000000000000068FFB4
:42C0D80000000000012001000000000000000000000120010000000810010A0048000000000000000000000000000000000000000000000000000000000000000000000054FD26
:42C11A00000000000000000000000000000000000000000000000000100002000000000000000000000000000000000000000000000000000000000000000000000000003CFD98
:42C15C00000000000000000000000000000000000000000000000000000000000000000000000000000000000000000000000000000000000000000000000000000000003CFE67
:42C19E00000000000000000000000000000000000000000000000000000000000000000000000000000000000000000000000000000000000000000000000000000000003CFE25
:42C1E000000000000000000000000000000000000000000000000000000000000000000000000000000000000000000000000000000000000000000000000000000000003CFEE3
:42C2220000000000000000000000000000000000000000000000000800000000000000000000000000000000000000000000000000000000000000000000000000000000B4FE20
:42C26400000000000000000000000000000000000000000000000000000000000000000000000000000000000000000000000000000000000000000000000000000000003CFE5E
:42C2A600000000000000000000000000000000000000000000000000000000000000000000000000000000000000000000000000000000000000000000000000000000003CFE1C
:42C2E800000000000000000000000000000000000000000000000000000000000000000000000000000000000000000000000000000000000000000000000000000000003CFEDA
:42C32A00000000000000000000000000000000000000000000000000000000000000000000000000000000000000000000000000000000000000000000000000000000003CFE97
:42C36C00000000000000000000000000000000000000000000000000000000000000000000000000000000000000000000000000000000000000000000000000000000003CFE55
:42C3AE00000000000000000000000000000000000002000000000000000000000000000000000000000000000000000000000000000000000000000000000000000000003CFC13
:42C3F00000000000000000000000000000000000000000000000000008100000000000000000000000000000000000000000000000000000000000000000000000000000ACFE49
:42C43200000000000000000000000000000000000000000000000000000000000000000000000000000000000000000000000000000000000000000000000000000000003CFE8E
:42C47400000000000000000000000000000000000000000000000000000000000000000000000000000000000000000000000000000000000000000000000000000000003CFE4C
:42C4B6000004010000000000000000000000000000000000000000000000000000000000000000000000000000000000000000000000000000000000000000000000000038FF08
:42C4F800000100000000000000000000000000000000000000000000000000000000000000000000000000000000000000000000000000000000000000000000000000002CFFD6
:42C53A00000000000000000000000000000000000000000000000000000000000000000000000000000000000000000000000000000000000000000000000000000000003CFE85
:42C57C00000000000000000000000000000000000000000000000000000000000000000000000000000000000000000000000000000000000000000000000000000000003CFE43
:42C5BE000017E002A8000950012A4005A8002DA0025C800B50012A4005A80015400200000000000950012A4005F80115A00254800A50012A800450011240054800092001E8FC60
:42C60000800C9001100106880011200244804010013240068800112002448008800100000000000688001120026482081001224004880011000320020C8008300006C00060FCAA
:02C64200FFFFF8
:00000001FF
